:100000000C94F2020C942A030C942A030C942A03F5
:100010000C942A030C942A030C942A030C942A03AC
:100020000C942A030C942A030C946A160C941F1542
:100030000C9404180C942A030C942A030C942A039D
:100040000C942A030C942A030C942A030C942A037C
:100050000C942A030C94C3170C942A030C942A03BF
:100060000C942A030C942A030C942A030C942A035C
:100070000C942A030C942A030C942A030C942A034C
:100080000C942A030C942A030C942A030C942A033C
:100090000C942A030C942A030C942A030C942A032C
:1000A0000C942A030C942A030C942A039D089D089F
:1000B000CF08CF0841095D09F40AF40A6809460A25
:1000C000570A570A20274727DF284727DF288F2787
:1000D000B227DF28A128B42800AD9DBD00AC9CBC90
:1000E00000AB9BBB00AA9ABA00A999B900A898B81E
:1000F00000A797B700A696B600A595B500A494B43E
:1001000000A393B300A292B200A191B100A090B05D
:10011000007D6D8D007C6C8C007B6B8B007A6A8A15
:100120000079698900786888007767870076668635
:100130000075658500746484007363830072628255
:100140000071618100706080004D3D5D004B3B5B44
:10015000004A3A5A00493959004838580047375739
:100160000046365600453555004434540043335359
:10017000004232520041315100403050001C0C2CE2
:10018000001A0A2A00190929001808280017072749
:100190000016062600150525001404240013032369
:1001A000001202220011012100100020001E0E2E5C
:1001B000004C3C5C001B0B2B004E3E5E001F0F2FC3
:1001C000004F3F5F007F6F8F00AF9FBF165C1E0028
:1001D0001F0020002100220023002400250026000B
:1001E00027002D002E002A002B0014001A00080002
:1001F000150017001C0018000C00120013002F003F
:1002000030003100396104001600070009000A00BF
:100210000B000D000E000F0033003400000028001A
:10022000E1001D001B000600190005001100100070
:10023000360037003800E50000000000E000E30071
:10024000E200000000002C00000000000000E600BA
:10025000015102510000E400165C3A003B003C00F2
:100260003D003E003F00400041004200430044008A
:1002700045004C0001000100520001000100010096
:10028000B200010049000100460047004800005C40
:100290000100500051004F00010001000100010069
:1002A000010001004A004B0000000100AC00AA0060
:1002B000A900A80001000100145C010001004D002C
:1002C0004E00AB0000000000010001000100000032
:1002D000000001000000000000000100010001001A
:1002E0000000010001003A003B003C003D003E00E0
:1002F0003F004000410042004300440045004C00E4
:100300000100C35C0100C65CC75CC85CC95CCA5C18
:10031000CB5CC45C010001000100005C0100010035
:10032000010001000100010001000100CC5CCD5C76
:1003300001000100000001000100010001000100B6
:1003400001000100010001000100010001000100A5
:100350000000000001000100010000000000010099
:100360000000000000000100010001000000010089
:1003700005010902A10185020901A1000509190170
:10038000290815002501950875018102050109302C
:1003900009311581257F9502750881060938158177
:1003A000257F950175088106050C0A3802158125FF
:1003B0007F950175088106C0C005010980A10185EE
:1003C0000319012AB700150126B7009501751081A0
:1003D00000C0050C0901A101850419012AA002151C
:1003E0000126A002950175108100C005010906A132
:1003F000018506050719E029E7150025019508750F
:100400000181020507190029EF1500250195F075F6
:1004100001810205081901290595057501910295CB
:100420000175039101C005010906A101050719E045
:1004300029E71500250195087501810295017508C8
:1004400081010507190029FF150026FF0095067593
:100450000881000508190129059505750191029586
:100460000175039101C009023B00020100A0FA09D5
:1004700004000001030101000921110100012240D3
:1004800000070581030800010904010001030000C1
:100490000009211101000122B60007058203200096
:1004A0000112010002000000085A4421120200015A
:1004B0000200011A0344005A00360030005200477F
:1004C0000042005F0041004E005300490000000E52
:1004D0000344005A00540045004300480000000453
:1004E00003090400010101010101010101020202ED
:1004F00002020202020203030303030303030404D0
:100500000404040404050505050506060606060799
:100510000707070708080808090909090A0A0A0B52
:100520000B0B0C0C0C0D0D0D0E0E0E0F0F0F1010F3
:10053000111111121213131414151516161717187A
:100540001819191A1A1B1B1C1D1D1E1E1F202021E5
:100550002222232424252626272829292A2B2C2D2C
:100560002D2E2F30313232333435363738393A3B4D
:100570003C3D3E3F404142434445464748494A4C42
:100580004D4E4F50515354555658595A5B5D5E5F0E
:10059000616264656668696B6C6D6F7072737577A4
:1005A000787A7B7D7E8082838587888A8C8E8F9106
:1005B000939596989A9C9EA0A2A3A5A7A9ABADAF30
:1005C000B1B3B5B7BABCBEC0C2C4C6C9CBCDCFD11A
:1005D000D4D6D8DBDDDFE2E4E7E9EBEEF0F3F5F8C3
:1005E000FAFDFF0011241FBECFEFDAE0DEBFCDBF62
:1005F00004B603FE18C080912F0690913006A0919A
:100600003106B09132068730904BA740B04B59F479
:1006100010922F0610923006109231061092320678
:10062000E0E0F8E3099512E0A0E0B1E0E8E9F2E6E5
:1006300002C005900D92A636B107D9F726E0A6E6CE
:10064000B2E001C01D92AF32B207E1F70E94E21F93
:100650000C944A310C9400002EE0929F800D1124DE
:10066000682F669566956695982F977085E0689FC8
:10067000B001112440E050E080E0FB01E40FF51FE1
:10068000E759FD4F208130E0092E02C036952795AD
:100690000A94E2F721703327042E01C0220F0A9436
:1006A000EAF7822B4F5F5F4F4530510531F70895D0
:1006B0002EE0929F800D1124E82FE695E695E695B1
:1006C000877051E001C0550F8A95EAF785E0E89FF1
:1006D000F0011124E759FD4F20E030E070E0408147
:1006E000CB01022E02C0969587950A94E2F781709D
:1006F000819584278523842781932F5F3F4F253061
:10070000310569F7089580E090E00E94A01880E02C
:1007100090E00E948A18109250050E943F1CEBEF57
:10072000F5E086E0DF011D928A95E9F71092F50564
:100730001092F4051092F6050C947C2D60936405DC
:100740007093650580936605909367050C94830309
:100750000F931F9341E050E060E070E004C0440F4D
:10076000551F661F771F8A95D2F780916405909177
:100770006505A0916605B09167058A019B01082B6C
:10078000192B2A2B3B2BC901B8011F910F910C94F7
:100790009E038F929F92AF92BF92DF92EF92FF9251
:1007A0000F931F93CF93DF9380906405909065051E
:1007B000A0906605B090670540915305509154058F
:1007C0006091550570915605842A952AA62AB72A64
:1007D000CFE1D0E02EE0929F7001112496E4D92E53
:1007E000082F10E0D501C4010C2E04C0B695A795C2
:1007F000979587950A94D2F780FD04C0219790F7CA
:1008000080E014C0DC9EF001DD9EF00D1124EE0DA1
:10081000FF1DE00FF11FEE0FFF1FE453FE4F859108
:1008200094910E941C1A019749F38C2FDF91CF916C
:100830001F910F91FF90EF90DF90BF90AF909F902E
:100840008F9008950F931F9341E050E060E070E0B7
:1008500004C0440F551F661F771F8A95D2F7409535
:100860005095609570958091640590916505A09173
:100870006605B09167058A019B01082319232A2385
:100880003B23C901B8011F910F910C949E03609303
:1008900053057093540580935505909356050C9419
:1008A0008303FC01808191810E94441D92959F7079
:1008B000963079F010F4925001C09A50923068F45A
:1008C000803F69F018F4883E40F409C0843F29F461
:1008D00006C0883E20F0813F11F080E0089581E05D
:1008E00008951092510580911001882331F0809174
:1008F000D10487FF02C08EE101C086E0E9EDF4E09B
:10090000DF011D928A95E9F70C948303882321F077
:100910000E94381C0C943F1C0895882339F0909154
:100920005105892B809351050C943F1C0895882311
:1009300079F19CEF980F913A30F4682F87ED94E0AD
:100940000E942D180DC090E2980F983058F48770CF
:1009500091E001C0990F8A95EAF7892F0E94381C0F
:100960000C943F1C9BE5980F933020F480E090E0BE
:100970000C94A01898E5980F973120F480E090E04F
:100980000C948A188D3E20F00E94682C0C947C2DCB
:100990000895CF93882309F472C0C82F8CEF8C0F71
:1009A000813AC0F5809110018823E1F08091D10453
:1009B00087FF18C0EC2FE695E695E695F0E0E95242
:1009C000FB4F8281282F30E04C2F477081E090E070
:1009D00002C0880F991F4A95E2F782239323892B3F
:1009E00061F412C0E9EDF4E08FED94E02191C217BB
:1009F00021F08E179F07D1F707C06C2F87ED94E089
:100A00000E942D180E943F1C6C2F87ED94E00E94DD
:100A1000551810C080E28C0F883078F4C77081E0E0
:100A200090E001C0880FCA95EAF790915105892B93
:100A300080935105CF910C943F1CEBE5EC0FE33014
:100A400040F4F0E0E45EFE4F808190E0CF910C94A2
:100A5000A018E8E5EC0FE73150F4F0E0EE0FFF1FCF
:100A6000E15EFE4F80819181CF910C948A18CD3E3A
:100A700030F08C2F0E94212DCF910C947C2DCF91A2
:100A800008951F93CF93DF93CDB7DEB767970FB667
:100A9000F894DEBF0FBECDBF4B8B5C8B6D8B7E8B16
:100AA0008F8B61111092500586E09E01235F3F4FAE
:100AB000D901E82F1D92EA95E9F795E0FE017396BA
:100AC000D90101900D929A95E1F79C894E895F8931
:100AD0007B897D879E876F87598B488BF901DE0163
:100AE000179601900D928A95E1F7CE0107960E9424
:100AF000601D81113EC086E0FE013796DE01119631
:100B000001900D928A95E1F7FF81E8856A857B85E2
:100B10006115710531F0EF3F31F481E0FF3F19F4C9
:100B200003C081E001C080E080FD23C02091FD046E
:100B300030E0C90101968770992740912E0550E059
:100B40008417950779F1F983EA837D836C8396E0B6
:100B5000929FD001939FB00D1124A250BB4FFE0174
:100B6000319601900D929A95E1F78093FD040E94D1
:100B7000CE1C16E080912E059091FD048917F9F0A6
:100B8000189FC001112482509B4F0E94601D882332
:100B9000B1F080912E0590E001968770992780939F
:100BA0002E05E8CF0E9471041092FD0410922E05CC
:100BB000E7EFF4E086E0DF011D928A95E9F767969A
:100BC0000FB6F894DEBF0FBECDBFDF91CF911F915E
:100BD00008958F929F92AF92BF92CF92DF92EF9241
:100BE000FF920F931F93CF93DF93CDB7DEB72A9772
:100BF0000FB6F894DEBF0FBECDBFFC010081D180DF
:100C000083819481892B39F01FEFD11206C091E0C6
:100C10000F3F19F403C091E001C090E090FDC0C502
:100C20007F0185E0DE01169601900D928A95E1F72D
:100C3000F70122818E819F81222349F00E94C903FE
:100C4000182F682F8E819F810E94580303C00E9435
:100C50002C03182F26E4129FF00111243EE0D39EAE
:100C6000E00DF11D1124E00FF11DEE0FFF1FE45305
:100C7000FE4F05911491043F8CE5180759F190F44B
:100C8000093DECE51E07E9F00A3DFCE51F07A1F16F
:100C9000083D2CE51207B1F506E221EE41EE68EDC4
:100CA0007CE514C0063F3CE5130701F1C8F0073F9F
:100CB0009CE5190739F507E225EE46EE67EF7CE57E
:100CC00005C007E225EE45EE69ED7CE5C7010E940F
:100CD000C218E5C406E221EE40EE64EF7CE5F6CFF3
:100CE00007E225EE44EE65EF7CE5F0CF06E221EE6B
:100CF00042EE66EF7CE5EACF08E221E045EE6AEDE0
:100D00007CE5E4CFF7018281882309F45BC110926E
:100D1000C5040430FDE51F0758F40B3F2CE512070E
:100D200080F4C80182509C45449708F035C109C041
:100D300002363DE5130729F0063A8DE5180709F05C
:100D40002BC10E94B61B9093D2048093D104013131
:100D50009CE5190709F4C6C008F042C00930FCE55B
:100D60001F0709F49BC000F505303CE5130709F4A3
:100D700085C078F403309CE5190709F478C008F0C1
:100D80007AC002301C4509F0F7C08091D10481601F
:100D9000F1C007302CE5120709F478C008F07AC0DA
:100DA0008091D1048061E6C00D308CE5180709F40C
:100DB00087C058F40B30ECE51E0709F479C008F041
:100DC0007BC08091D10488606FC00F302CE5120782
:100DD00009F480C008F082C08091D104877FCAC026
:100DE0000E3F8CE5180709F471C000F50531ECE5FC
:100DF0001E0709F485C068F403312CE5120709F4D5
:100E000075C008F095C00E9471048091D1048F775D
:100E1000B1C00C3F8CE51807A9F108F054C00B3F96
:100E20001C4509F0A9C08091D20440C00230FDE504
:100E30001F0709F489C058F401153DE5130709F4AB
:100E40005AC008F069C08091D20482602FC0023677
:100E50009DE5190709F47EC0063AEDE51E0709F481
:100E600083C003301D4509F087C060E06EC08091EB
:100E7000D10482607FC08091D10416C08091D104DA
:100E8000886078C08091D20482604FC08091D10484
:100E9000806270C08091D10480646CC00E94710433
:100EA0008091D104806866C0846064C081603DC068
:100EB0008091D1048E7F5EC08091D1048D7F5AC015
:100EC0008091D10416C08091D20418C08091D204C0
:100ED0008D7F2BC08091D1048F7E4CC08091D10436
:100EE0008F7D48C08091D1048F7B44C08091D10414
:100EF000877F8B7F3FC08091D2048D7F8E7F15C00E
:100F00008091D10482FB222720F991E0922790FB67
:100F100082F990FB83F92EC08091D204982F90958E
:100F200091708E7F892B90FB81F98093D20424C02D
:100F30000E9471048091D10487FB222720F991E05F
:100F4000922790FB87F916C061E08EE090E00E9446
:100F5000933012C08091D10484FB222720F991E0C4
:100F6000922790FB84F906C08091D104982F909528
:100F700090FB80F98093D1046091D1041091D20448
:100F800084E090E00E949330612F82E290E00E9422
:100F900093300E94710483C306312CE5120721F5BA
:100FA000809151058A7A91E009F490E0909368026B
:100FB000882311F065E301C069E287ED94E00E94A7
:100FC00055180FC00631FCE51F0709F040C080919D
:100FD0006802882309F486C365E387ED94E00E94E4
:100FE0002D180E943F1C5BC30B35FDE51F0749F11F
:100FF00058F401153CE51307B1F00F3D1C4509F00D
:1010000040C00E94C71B4BC30C359DE51907D9F0A2
:101010000D351D45B1F58091D20482FB882780F9FA
:1010200091E0892711C00E947104FFEF04E31CE0E6
:10103000F15000401040E1F700C000000E949F17EF
:101040002EC381E001C080E00E94B11C1AC08091D3
:10105000510582720B3C2CE5120709F48AC308F48F
:1010600000C3003D3CE5130709F496C308F44EC3E2
:10107000073D8CE5180708F458C30E351D4509F4E3
:101080000EC3F70182810081D180882359F0802F1F
:101090009D2D0E94C903182F682F802F9D2D0E941F
:1010A000580305C0802F9D2D0E942C03182F26E485
:1010B000129FF00111243EE0D39EE00DF11D11249A
:1010C000E00FF11DEE0FFF1FE453FE4F8591949149
:1010D0000E941C1A8C01982EF701D280A580A29440
:1010E0003FE0A32280912F058770B9F0DD20A9F0A1
:1010F000812F807F803421F080E2800F883068F07B
:101100008091D20482FD09C082E00E94941C8091EB
:101110002F058770CC24C3948111C12CB12EB294B9
:101120009FE0B9228B2D90E08C30910508F05CC2D5
:10113000FC01EA5AFF4F0C942E31812F807F1F70E3
:10114000882311F01295107FDD20B9F0112309F4E6
:1011500038C280E2800F883010F0911006C0809174
:101160005105182B1093510505C080915005182B7F
:10117000109350050E943F1C24C2802F0E949704A8
:10118000112309F431C2005E083078F1992069F129
:1011900010958091500518231093500529C0812F78
:1011A000807F1F70803211F01295107F992021F0FE
:1011B000F1E09F16D9F149C08091D20482FF1BC093
:1011C000DD2069F0112339F080915105182B10931F
:1011D00051050E943F1C80E00E94C90405C280E0C6
:1011E0000E949704112309F4FFC1812F0E94381C2B
:1011F0000E943F1CF9C1DD2081F080915205AA2098
:1012000051F001E0A01207C0182B181709F4ECC127
:1012100010935205E9C1812B10C0AA2021F021E0D2
:10122000A21609F4E1C10E94321C27C0DD2041F062
:1012300035E03A1508F4D8C1812F0E948D04D4C13D
:1012400084E08A1508F4D0C118C0DD2049F0AA2036
:1012500099F3F701858180FFB4C18F708583ECCF4E
:10126000AA2059F0093309F0BCC1FFEF17EE23E0C3
:10127000F15010402040E1F7B2C1812F0E94860456
:10128000B3C1812F86958695837019F0813059F00E
:10129000ABC1DD2019F0C801937002C080E090E07E
:1012A0000E94A018A7C1DD2019F0C801937002C0E8
:1012B00080E090E00E948A189DC1802FDD2019F007
:1012C0000E94212D02C00E94682C0E947C2D92C198
:1012D000812F837009F069C0D1108AC1902F929537
:1012E00096959770990F990F802F8F70882E912C5B
:1012F000A12CB12C092E04C0880C991CAA1CBB1C63
:101300000A94D2F704FF12C04FE050E060E070E0B2
:1013100004C0440F551F661F771F9A95D2F7DB0153
:10132000CA0180959095A095B09503C080E090E0AB
:10133000DC0116951695412F4370423019F1C8F41F
:101340000091530510915405209155053091560593
:10135000413059F088299929AA29BB29BC01CD011E
:1013600060237123822393230AC0802A912AA22A10
:10137000B32ABC01CD01682979298A299B290E94B9
:10138000470436C188299929AA29BB290091530508
:10139000109154052091550530915605BC01CD01A1
:1013A0006027712782279327EACFDD2019F0812F4C
:1013B000817001C08695882309F41AC1902F9295F7
:1013C00096959770990F990F802F8F70882E912C7A
:1013D000A12CB12C092E04C0880C991CAA1CBB1C82
:1013E0000A94D2F704FF12C04FE050E060E070E0D2
:1013F00004C0440F551F661F771F9A95D2F7DB0173
:10140000CA0180959095A095B09503C080E090E0CA
:10141000DC0116951695412F43704230D9F068F5DE
:10142000009164051091650520916605309167056E
:10143000413059F088299929AA29BB29BC01CD013D
:1014400060237123822393231EC0802A912AA22A1B
:10145000B32A13C088299929AA29BB2900916405B8
:10146000109165052091660530916705BC01CD019D
:10147000602771278227932706C0BC01CD01682908
:1014800079298A299B290E949E03B2C01F70DD2002
:1014900039F0812F0E94A803802F0E948D04A8C0DC
:1014A000802F0E948604812F0E942204A1C0802FD9
:1014B00032EF931609F443C0391538F090EF9916BE
:1014C00059F0E1EF9E16B1F177C0F3EF9F16F1F1FD
:1014D00024EF921659F170C0DD2019F134E03A156D
:1014E00008F482C01F7181E090E0A0E0B0E0AC01A0
:1014F000BD0104C0440F551F661F771F1A95D2F710
:101500008091640590916505A0916605B09167058D
:101510008A019B01082719272A273B27C901B801FF
:1015200029C025E02A1508F45FC0DCCF8091D204E1
:1015300082FF23C0DD2029F0812F8F7130C0DD2094
:10154000D9F3812F8F710E9422044EC0DD2079F0E3
:101550001F7181E090E0A0E0B0E0BC01CD0104C0CB
:10156000660F771F881F991F1A95D2F703C060E096
:1015700070E0CB010E949E0337C0DD2099F01F71FF
:10158000812F0E94A8038091D20482FD07C038E019
:10159000139FC0011124836080932F05812F0E9427
:1015A000A80322C081E00E94941C81E08A15E0F427
:1015B00082E00E94941C18C0DD2029F0AA2009F4C2
:1015C000BBCF802F09CEAA2009F4BBCF893349F4C1
:1015D0009FEFE7EEF3E09150E040F040E1F700C00C
:1015E0000000802F0E94970488EF8B0D843010F448
:1015F0000E94B618CC20A9F080912F0580FD11C063
:10160000F70112828595859585950E94A803C701EB
:101610000E94E90580912F058595859585950E9405
:10162000220485E0F701DE01119601900D928A9562
:10163000E1F789819A810E942C039A8106E4809FB8
:10164000F00111241EE0919FE00DF11D112489810C
:10165000E80FF11DEE0FFF1FE453FE4F85919491AB
:101660009FC0063C9CE5190709F46FC0E8F5043CEF
:10167000FCE51F0709F45FC008F062C0033C1C458D
:1016800009F0FFCC9091EE0581E089278093EE056B
:10169000109211018091C00581608093C0058091F6
:1016A0002F05877009F47CC0F7018281882309F433
:1016B00077C08091D20482FD73C082E02A960FB673
:1016C000F894DEBF0FBECDBFDF91CF911F910F9178
:1016D000FF90EF90DF90CF90BF90AF909F908F9052
:1016E0000C94941C69E279CC083C9CE51907B9F18B
:1016F00088F1093CFCE51F07B9F10A3C1C4509F0DB
:10170000C0CC42EC5DE26EEC7DE241C00D3CECE50C
:101710001E07C9F198F10E3C2CE51207D9F10F3CD8
:101720001C4509F0AECC84E038C0023D1C4508F0F1
:10173000B6CF8EE032C044E05EE26DE07EE227C0CC
:101740004DE05EE264E07EE222C042EF5DE26BEFDC
:101750007DE21DC04BEF5DE262EF7DE218C04AED15
:101760005DE266EE7DE213C046EE5DE26AED7DE28B
:101770000EC04EEC5DE262EC7DE209C046EA5DE23D
:1017800064EB7DE204C044EB5DE266EA7DE20E9428
:101790004D1985CF81E001C089E00E94D2257FCF1D
:1017A0002A960FB6F894DEBF0FBECDBFDF91CF9162
:1017B0001F910F91FF90EF90DF90CF90BF90AF906F
:1017C0009F908F9008952F923F924F925F926F92C9
:1017D0007F928F929F92AF92BF92CF92DF92EF92C1
:1017E000FF920F931F93CF93DF93CDB7DEB72E9762
:1017F0000FB6F894DEBF0FBECDBF182F8091180131
:1018000081130DC02091EE05237030E04091170147
:1018100050E081E02417350719F480E001C081E031
:101820008170809314018091F305909113019817B2
:1018300039F08093130140E060E080E00E94C02A0C
:10184000103109F04CC085E999E205C0133108F068
:101850008FC283E699E20E949924082F2CC0183089
:1018600008F095C1133009F44BC008F0F6C01130F0
:1018700009F090C0809112010DE0809F002D11248D
:10188000ADE0FA2EF00E2DE32F1510F4FDE3FF2E40
:101890006091EF057091F0058091F1050E94D82BC1
:1018A000E62ED72EC82E0F1508F481C001E03CE3C8
:1018B0003F1508F47AC0809112018F5F8093120166
:1018C0000111A0C682E08093110180911401811161
:1018D00099C6111197C683E08093110193C6113107
:1018E00008F081C1173009F0BACF85E89AE205C047
:1018F0001D3008F062C183EC99E20E94FA24ADCF5A
:10190000009112018DE0089F002D11246DE0D62E6C
:10191000D00EADE3AD1510F45DE3D52EB090F0051B
:10192000A090F1052091F20540E4C42E3C2D329F99
:10193000312D1124C32E0D1538F5E02EF12CF701B1
:10194000E05EFD4F9081809113018923D9F0F7016A
:10195000EE0FFF1FEA55FE4F6081C69EB0011124B5
:1019600035E0759567953A95E1F78091EF05680F39
:101970007B2D8A2D0E94D82B462F282F672FC70139
:101980000E94C22A0F5FD7CF01E08CE38D1508F0CB
:1019900092CF0BC01230E8F480911401882329F013
:1019A00040E060E080E00E94C02A00E084CFE02FA9
:1019B000F0E0DF01A05EBD4F8C9190911301982360
:1019C00031F02C2D4E2D6D2DCF010E94C22A0F5FBC
:1019D0006ACF009112018DE0089F002D1124EDE0E7
:1019E000FE2EF00E8DE38F1510F47DE3F72ED090D0
:1019F000F005E090F105C090EF05B6018E2D0E9434
:101A0000D82BB62EA72E982E6091F2056C0D7D2D49
:101A10008E2D0E94D82BE62ED72EC82E0F15B8F487
:101A2000802F90E0FC01E05EFD4F3081209113019A
:101A3000232359F030FF04C02C2D4E2D6D2D03C0F3
:101A4000292D4B2D6A2D0E94C22A0F5FE7CF01E09E
:101A50009CE39F1508F02FCFA8CF153059F481E0F3
:101A60009AE205C01A3008F09FC08FEF99E20E94F9
:101A70004B24F3CE163008F047C0009112018DE0E0
:101A8000089F002D11249DE0F92EF00E9DE39F1577
:101A900010F48DE3F82ED090EF05E090F005C090A3
:101AA000F1056091F2056695669566958091C10590
:101AB0009091C2050E94BB2B0E94072B805887FD86
:101AC0008195880F282F3C2D239F212D1124822FB3
:101AD0006D2D7E2D0E94D82BE62ED72EC82E0F15E9
:101AE00008F04FC0E02FF0E0DF01A05EBD4F8C9109
:101AF00090911301982331F02C2D4E2D6D2DCF0197
:101B00000E94C22A0F5FEBCF81EA9AE20E947625FB
:101B1000A4CE173108F08AC1009112018DE0089F10
:101B2000002D11247DE0F72EF00E3DE33F1510F45B
:101B30006DE3F62ED090F005E090F105C090EF0532
:101B40006091F2056695669566958091C1059091C4
:101B5000C2050E94BB2B0E94072B805887FD8195F0
:101B6000880F682F2CE0629F612D11246C0D7D2D54
:101B70008E2D0E94D82BE62ED72EC82E0F1508F4D6
:101B800043C101E08CE38F1508F095CE0ECF1B30DA
:101B900019F482ED99E26BCF1C3048F4193009F04A
:101BA00061CF86EF99E263CF8DEE99E260CF1D3071
:101BB00009F09ECE82E99BE2A9CF1E3019F484E79A
:101BC0009AE2A4CF1F3049F480E69AE296CE1F3104
:101BD00009F458C41F3F09F4E4C4809112018F5FD7
:101BE000809312016FCE183109F06DC040919602BA
:101BF0005091970260919802709199028091C1056D
:101C00009091C205A091C305B091C40584179507B2
:101C1000A607B70708F4C9CE0E944C2B082F0E94D4
:101C20004C2B9DE3891BF0F7890FE82EF12CF7016F
:101C3000E05EFD4F909113018081892309F441C03A
:101C400001FF04C020E040E060E013C00E944C2B84
:101C5000082F0E944C2B8695782F2FE7720F08F4DF
:101C60007FEF602F8091F1050E94D82B462F282FFF
:101C7000672FC7010E94C22A2091F20530E1230F8D
:101C800008F42FEF60E1822F90E00E94BB2BBC0193
:101C900084EF91E00E94EC2F8091C1059091C205E4
:101CA000A091C305B091C405860F971FA11DB11D5A
:101CB0008093960290939702A0939802B093990212
:101CC00074CE01E0F8CD193108F0B3C0143109F039
:101CD00046C08091140181111EC06091F20520E17F
:101CE000620F08F46FEF8091C1059091C2050E94C8
:101CF000BB2B65E070E00E94EC2F892B09F055CEDC
:101D00000E944C306DE370E00E941A316091130123
:101D10000E9453194ACE809112019DE0899F802D27
:101D20001124FDE0DF2ED80EEDE3ED1510F4EDE308
:101D3000DE2EE82EF12CAD2CB12CEA14FB044CF471
:101D400060911301C7010E945319FFEFEF1AFF0AB8
:101D5000F4CF01E02CE32D1508F0ADCD26CE1531E2
:101D600008F04CC0123109F071CD85E299E273CDD3
:101D70008091140181111EC06091F20520E1620F73
:101D800008F46FEF8091C1059091C2050E94BB2BB2
:101D90006AE070E00E94EC2F892B09F006CE0E94C9
:101DA0004C306DE370E00E941A31609113010E9483
:101DB0007A19FBCD809112019DE0899F802D11241D
:101DC000BDE0DB2ED80E9DE39D1510F4ADE3DA2EB9
:101DD000E82EF12CAD2CB12CEA14FB044CF46091EC
:101DE0001301C7010E947A19AFEFEA1AFA0AF4CF79
:101DF00001E0BCE3BD1508F05ECDD7CD163109F08A
:101E000088CE88E29BE233CEE02FF0E0DF01A05ED7
:101E1000BD4F8C9190911301982331F02C2D4E2DB4
:101E20006D2DCF010E94C22A0F5FA8CE84E199E2F6
:101E30001ECE1C3109F09BC080911401882371F0E3
:101E400040E060E080E00E94C02A86E4E3EAF3E03C
:101E5000DF011D928A95E9F71092A20363EAC62E6C
:101E600063E0D62E712C66246A9470EDA72EB12CF7
:101E7000E0EC5E2EFFE28F2E912C760100E0011146
:101E80000CC08091A203811108C00E944C3085359E
:101E900095401CF4F601608206C0D7018C918150F8
:101EA0008E3F08F48C93AE014F5F5F4F672D802FFC
:101EB0000E94C42A882309F1F7012081E981213D8C
:101EC00070F030E0205D3109529EC001539E900DAC
:101ED0001124B4010E94EC2F262F4FEF0AC0FFEF10
:101EE0002F9FC0011124B5010E94EC2F462F20E046
:101EF00060E08E2F90E00E94C22A0F5F2EE0E20E7B
:101F0000F11C053009F0BBCF73943FEFC31AD30A1D
:101F10008EE07812B2CF8091A2038F5F8D3118F4DA
:101F20008093A20342CD1092A2032DEC33E084E013
:101F30004EEFA3EAB3E0F9019EE0843041F4D89675
:101F40005C91D8975F3F19F4D8964C93D8975081FD
:101F50005F3F11F44083568791503196119691114D
:101F6000ECCF81502E5031098111E3CF1ECD1D31B0
:101F700008F07BC21A3109F0D4C040919B03509104
:101F80009C0360919D0370919E038091C105909187
:101F9000C205A091C305B091C40584179507A60793
:101FA000B70708F402CD80911401882329F040E09E
:101FB00060E080E00E94C02A6091EF057091F0051A
:101FC0008091F1050E94D82B062F772E682E85E58B
:101FD000C82E83E0D82E90E6E92E91E0F92E26EA6D
:101FE000422E21E0522E4601A12CB12CF401808119
:101FF000F701EA0DFB1D882329F08081262D402F53
:10200000672D04C0808120E040E060E090E00E9405
:10201000C22AD40111968C91F40181934F01FFEFF4
:10202000AF1ABF0A26E0A216B10401F74701560114
:10203000BDE03B2ED5011D968C91882331F0F40133
:102040008585262D402F672D06C0D4011D968C91C5
:1020500020E040E060E090E00E94C22AF501848523
:1020600085873A94F1E0AF1AB10821E0821A91080D
:1020700037E03312DFCFD60117968C91882331F0E9
:10208000F7018781262D402F672D06C0D7011796AF
:102090008C9120E040E060E090E00E94C22AF601CE
:1020A0008681882339F0D70116968C91262D402FF2
:1020B000672D05C0F701868120E040E060E090E0F8
:1020C0000E94C22A0E944C2B837091E009F090E09C
:1020D000D60116969C93169717969C93BEE0CB0E4E
:1020E000D11CEEE0EE0EF11C4E145F0409F07BCF24
:1020F0000E94C52BC090C105D090C205E090C305D9
:10210000F090C405DC01CB018C0D9D1DAE1DBF1DE3
:1021100080939B0390939C03A0939D03B0939E0395
:1021200044CC1B3108F0F4C040915103509152034C
:1021300060915303709154038091C1059091C20541
:10214000A091C305B091C40584179507A607B707EA
:1021500008F42BCC80911401811110C080911201E0
:102160000DE0809F002D11245DE0E52EE00E9DE343
:102170009E1508F05AC04DE3E42E57C040E060E0E1
:1021800080E00E94C02A3AE9C32E32E0D32EE12C2F
:10219000F12C0FE70E944C2B81FF08C0D6011C9246
:1021A00011961C92119712961C921CC00E944C2BE7
:1021B000982E0E944C2B8695782F700F08F47FEF95
:1021C000C701880F991F8E0D9F1DFC01E656FD4F1C
:1021D0005F01692D8091F1050E94D82BD5016D9387
:1021E0007D938C93BFEFEB1AFB0AE3E0CE0ED11C7C
:1021F000FDE3EF16F10471F6B1CFA02FB0E0FD01C1
:10220000E05EFD4F808190911301982369F0FD01FC
:10221000EE0FFF1FEA0FFB1FE656FD4F22814081A4
:102220006181CD010E94C22A0F5F0E1530F301E0DB
:102230002CE32E1508F400E03CE33E1508F03BCB00
:1022400020E0F12C81E0E81AF108822F90E08E1551
:102250009F05CCF4AC01440F551F480F591F46563B
:102260005D4F0196FC01EE0FFF1F8E0F9F1FFC01BB
:10227000E656FD4F80819181A281FA01808391838E
:10228000A2832F5FE2CF0E944C2B6701CC0CDD1C98
:1022900081FF0AC0C6018E0D9F1DFC01E656FD4F51
:1022A0001082118212821BC00E944C2BB82E0E94F9
:1022B0004C2B8695782F2FE7720F08F47FEFC6011D
:1022C0008E0D9F1D9C0126563D4F79016B2D8091EF
:1022D000F1050E94D82BD7016D937D938C930E94BA
:1022E000C52BC090C105D090C205E090C305F09009
:1022F000C405DC01CB018C0D9D1DAE1DBF1D80935F
:10230000510390935203A0935303B0935403D3CA41
:10231000809112010DE0809F002D1124FDE0F00F4F
:10232000F987F73410F026E4298780911401882377
:1023300061F040E060E080E00E94C02A86E4E3EAC9
:10234000F3E0DF011D928A95E9F780911201811176
:1023500015C08091A0039091A1030E94E91721E08C
:102360008931910508F420E020939F03499730F0CC
:102370000E94F8179093A1038093A003E02EF12C04
:10238000B9854B2E512CAEE03A2EFE0131964F010D
:10239000E414F5040CF063C0C70165E070E00E942E
:1023A0001A316B013C01389EF001399EF00D112469
:1023B000ED55FC4FE60FF71F0081A4010E94C42ACF
:1023C000282E54018A2D8819821508F031C0D501B4
:1023D000EC91F0E0E05EFD4F908180911301892344
:1023E00019F1302F25E5321B08F430E07091F0052B
:1023F0002AEA200F08F42FEF4091F10582E0289F90
:10240000200D11242E5F249F212D11246AEA631BC5
:10241000822F0E94D82B462FD5019C91282F672F01
:10242000892F90E00E94C22ABFEFAB1ABB0ACACF25
:1024300080919F03882379F021E0021B08F400E0DB
:10244000369CC001379C900D11248D559C4FFC018A
:10245000EC0DFD1D00833FEFE31AF30A99CF01E075
:102460008985863408F427CAA0CA1E3129F487E07A
:1024700099E20E94D623F1C91E3108F0A8CB8DE065
:1024800099E2F7CF5090C50521E0352D321B08F4B5
:1024900030E03A87D09012018DE0D89ED02C1124E4
:1024A0008D0D89878E33A0F09DE3998711C020910F
:1024B000F1053C2D329F312D1124832FB1010E9453
:1024C000D82B462F282F672FC3010E94C22AD394EE
:1024D0008985D81608F060C06D2C712CF301E05E80
:1024E000FD4F908180911301892389F32090EF059E
:1024F0003090F0054A84C12CC301880F991FDC017C
:10250000AA55BE4FBC87AB87C301880F991FFC013A
:10251000E955FE4FFE87ED87451448F6E42CF12C73
:10252000AB85BC85AC90B12CF701EB53FA4F8181A0
:10253000A81AB108AD85BE858C90912C8185881A2A
:102540009108AA9C9001AB9C300D300D1124889C01
:10255000C001899C900D900D1124820F931F0E9441
:10256000612B082F6091F20521E0620F08F46FEFF4
:10257000F701EE0FFF1FEB53FA4F818D928D0E94F2
:10258000BB2B7C019401A501B1018C2D0E94F12A85
:102590001B01C82E4394C0CF01E08D3308F48BC9D2
:1025A00004CA8091C1059091C205A091C305B09164
:1025B000C40588279C70AA27BB272AE0B695A79553
:1025C000979587952A95D1F782309105A105B10598
:1025D00071F083309105A105B10569F040E00197E4
:1025E000A105B10511F060E008C064E102C044E15A
:1025F00060E080E003C044E164E184E10E94C02A1D
:1026000082E06AC92E960FB6F894DEBF0FBECDBF2A
:10261000DF91CF911F910F91FF90EF90DF90CF90BE
:10262000BF90AF909F908F907F906F905F904F90F2
:102630003F902F900895089580917F05089580938D
:10264000D3047093D5046093D4048091A2058430A0
:1026500001F582E08093E9008FEF9091E8008150CE
:1026600095FD06C095ED9A95F1F700008111F5CF23
:102670008091E80085FF0DC040E050E063E070E02D
:1026800083ED94E00E940E268091E8008E7780937F
:10269000E8000895BC0184E00C941F13BC0183E0A2
:1026A0000C941F1322E02093E9002FEF3091E800F3
:1026B000215035FD06C035ED3A95F1F700002111A6
:1026C000F5CF2091E80025FF0BC040E050E066E028
:1026D00070E00E940E268091E8008E778093E800DB
:1026E0000895CF93DF9320911001222339F0209198
:1026F000D10427FF03C060E222E002C068E021E0CD
:102700002093E9002FEF3091E800215035FD06C0FD
:1027100035ED3A95F1F700002111F5CF2091E80051
:1027200025FF1DC0EC0180911001811105C040E022
:1027300050E068E070E003C070E040E050E0CE019F
:102740000E940E268091E8008E778093E80080E258
:10275000FE01A0E8B5E001900D928A95E1F7DF91C6
:10276000CF910895FF920F931F93CF93DF9300D0E3
:1027700000D0CDB7DEB78D33910568F5122F042F49
:10278000F62EBC01660F771F660F771F68527F4FCA
:1027900044E050E0CE0101960E945C308981837054
:1027A0002A81E82FF0E030EC839FC00111248D5F77
:1027B0009B4FDC01A20FB11DFC922B81DC01A20F0B
:1027C000B11D0C932C81DC01A20FB11D1C93EE5F97
:1027D000FB4F81E080830F900F900F900F90DF915F
:1027E000CF911F910F91FF900895FF920F931F9328
:1027F000CF93DF93182F062FF42EC0E0D0E02F2DBB
:10280000402F612FCE010E94B2132196CD33D10506
:10281000B1F7DF91CF911F910F91FF9008950F9322
:102820001F93CF9380910204882331F165EC8EEFE2
:102830000E94FB2561E08DEF0E94FB2503E014E080
:10284000C0E0C093AC05EDEAF5E0D8018D9181932D
:1028500085E0ED3BF807D1F724E630E041E150E0B8
:102860006CEA75E080EA0E94C52F892B59F4C05F9D
:10287000005F1F4FC03C29F710920204CF911F91B7
:102880000F91089581E080930104F6CFAF92BF923B
:10289000CF92DF92EF92FF920F931F93CF93DF932C
:1028A00000D000D0CDB7DEB70E940E2F65EC8EEFC2
:1028B0000E94FB2560E08DEF0E94FB2510E060E0A8
:1028C000812F0E94FB251F5F1831C9F765EC8EEF41
:1028D0000E94FB2561E08DEF0E94FB2510E060E087
:1028E000812F0E94FB251F5F103CC9F765EC8EEF1E
:1028F0000E94FB2563E08DEF0E94FB2560E08FE0E6
:102900000E94FB2560E080E10E94FB256FEF81E0E3
:102910000E94FB2561E080E00E94FB258FE39CE99B
:102920000197F1F700C0000008ED10E09CECC92E03
:1029300091E0D92E28E1A22EEE24E394F12CBB24C1
:10294000B39444E050E0B801CE0101960E945C309F
:102950006A815B814C818981837090E0762F7695C6
:1029600076957695A89E9001A99E300D1124275149
:102970003C4FF901E70FF11D6770D70102C0AA0FA4
:10298000BB1F6A95E2F7BD017081672B6083652FDD
:10299000669566956695F901E60FF11D5770B701CA
:1029A00001C0660F5A95EAF75081652B6083542F5A
:1029B000569556955695F901E50FF11D477097010B
:1029C00002C0220F331F4A95E2F7A9012081422B52
:1029D0004083FC01EF5FFB4FB0820C5F1F4FC016BE
:1029E000D10609F0AECF80910104811111C010927F
:1029F00001040F900F900F900F90DF91CF911F91D6
:102A00000F91FF90EF90DF90CF90BF90AF9008951F
:102A100065EC8EEF0E94FB2560E08DEF0E94FB25A8
:102A200089EEE82E83E0F82E10E0D7016D917D014C
:102A3000812F0E94FB251F5F1831B9F7D8CF1F9255
:102A40000F920FB60F9211242F933F934F935F93E2
:102A50006F937F938F939F93AF93BF93CF93DF93A6
:102A6000EF93FF93C091E900CF708091EC00D82FD5
:102A7000D17080FDD0E81092E9008091F000877F4E
:102A80008093F00078940E943A261092E900809199
:102A9000F00088608093F000CD2BCF70C093E900E8
:102AA000FF91EF91DF91CF91BF91AF919F918F9166
:102AB0007F916F915F914F913F912F910F900FBE3A
:102AC0000F901F901895E8EDF0E080818E7F808355
:102AD0001092E2001092DA001092E100A0EEB0E055
:102AE0008C9181608C9380818F77808319BCA7ED56
:102AF000B0E08C918E7F8C9380818F7E808310924A
:102B0000D60408952091E4003091E50095E64091C7
:102B1000EC00842F817040FF23C08091E80080FD8D
:102B20001DC08091A205882399F0853099F080918D
:102B3000EB0085FD11C04091E4005091E5002417A1
:102B4000350729F3915011F09A01E1CF84E00895FF
:102B500082E0089583E0089581E0089580E008957B
:102B60004091E80042FFDDCF08958091A40587FFE2
:102B700011C08091E80082FD05C08091A2058111FD
:102B8000F8CF11C08091E8008B770BC08091A2052F
:102B9000882349F08091E80080FFF8CF8091E80019
:102BA0008E778093E8000895982F973068F590937A
:102BB000E900981739F07091EC002091ED005091E8
:102BC000F00003C0242F762F50E021FD02C09F5F4C
:102BD000ECCF3091EB003E7F3093EB003091ED0075
:102BE0003D7F3093ED003091EB0031603093EB008E
:102BF0007093EC002093ED005093F0002091EE00D4
:102C000027FDE5CF80E008958F708093E90081E093
:102C10000895CF92DF92EF92FF920F931F93CF937D
:102C2000DF93C8EDD0E088818F7E8883E7EDF0E008
:102C300080818160808384E082BF81E08093D604BC
:102C400088818E7F888302EE10E0F8011082109256
:102C5000DA0081EEC82ED12CF601108288818F77A0
:102C6000888388818068888388818F7D888319BC68
:102C70001092A2051092A3051092A1051092A00532
:102C800090EEE92EF12CF70180818B7F8083888183
:102C90008160888342E060E080E00E94D415F60104
:102CA00080818E7F8083F801808181608083808134
:102CB00088608083F70180818E7F80838881806136
:102CC0008883DF91CF911F910F91FF90EF90DF905C
:102CD000CF9008951F920F920FB60F9211242F9349
:102CE0003F934F935F936F937F938F939F93AF9394
:102CF000BF93EF93FF938091E10082FF09C0809121
:102D0000E20082FF05C08091E1008B7F8093E100AB
:102D10008091DA0080FF2AC08091D80080FF26C011
:102D20008091DA008E7F8093DA008091D90080FF55
:102D300018C080E189BD82E189BD09B400FEFDCFE4
:102D400081E08093A2058091D60481110FC00E947A
:102D500063150E9409168091E20084608093E2006E
:102D600005C019BC1092A2051092D6048091E10012
:102D700080FF17C08091E20080FF13C08091E200C5
:102D80008E7F8093E2008091E20080618093E20078
:102D90008091D80080628093D80019BC85E0809330
:102DA000A2058091E10084FF30C08091E20084FFA1
:102DB0002CC080E189BD82E189BD09B400FEFDCF50
:102DC0008091D8008F7D8093D8008091E1008F7E24
:102DD0008093E1008091E2008F7E8093E2008091F9
:102DE000E20081608093E2008091A305882311F0C6
:102DF00084E007C08091E30087FD02C081E001C04C
:102E000083E08093A2058091A2058091E10083FF79
:102E100027C08091E20083FF23C08091E100877F7B
:102E20008093E10082E08093A2051092A305809137
:102E3000E1008E7F8093E1008091E2008E7F80939D
:102E4000E2008091E20080618093E20042E060E075
:102E500080E00E94D4158091F00088608093F0009B
:102E6000FF91EF91BF91AF919F918F917F916F9162
:102E70005F914F913F912F910F900FBE0F901F9038
:102E800018952091AA053091AB052617370748F011
:102E90006115710539F42091E8002E772093E80040
:102EA00001C0B901FC0120E06115710579F1809143
:102EB000A2058823F1F18530F1F18091E80083FDCE
:102EC0003CC08091E80082FD2EC08091E80080FF28
:102ED000EBCF2091F3008091F20090E0922B6115EE
:102EE000710551F08830910538F421912093F1005B
:102EF000615071090196F3CF21E0089709F020E0B5
:102F00008091E8008E778093E800CECF2111CFCF5B
:102F10000AC08091A205882361F0853061F080911C
:102F2000E80083FD0AC08091E80082FFF2CF80E0D4
:102F3000089582E0089583E0089581E0089581E096
:102F40008093E00080E28093D8001092C9008FE166
:102F50009EE40197F1F700C0000087E090EBDC01F0
:102F600080932F0690933006A0933106B0933206DB
:102F70009CE088E10FB6F894A895809360000FBE9E
:102F800090936000FFCF78941F920F920FB60F922C
:102F900011248F939F93AF93BF938091CD04909111
:102FA000CE04A091CF04B091D0040196A11DB11D13
:102FB0008093CD049093CE04A093CF04B093D0041B
:102FC000BF91AF919F918F910F900FBE0F901F9067
:102FD00018959C014FB7F8948091CD049091CE0440
:102FE000A091CF04B091D0044FBF821B930B0895E2
:102FF0002FB7F8948091CD049091CE04A091CF0486
:10300000B091D0042FBF08951F920F920FB60F9268
:1030100011248F939F93AF93BF938091CC04811120
:1030200013C08091CD049091CE04A091CF04B091B3
:10303000D0044196A11DB11D8093CD049093CE0480
:10304000A093CF04B093D004BF91AF919F918F9183
:103050000F900FBE0F901F90189520911001222302
:10306000C9F02091D10427FF15C0262F269526955B
:1030700026952E31C8F4FC01E20FF11D677081E046
:1030800090E001C0880F6A95EAF7809592818923C4
:1030900082830895FC0106962281621301C0128288
:1030A0003196E817F907C1F70895209110012223FE
:1030B000C1F02091D10427FF14C0262F2695269514
:1030C00026952E3130F5FC01E20FF11D677081E08D
:1030D00090E001C0880F6A95EAF79281892B82837C
:1030E0000895FC0132962FEF30E04191641789F08A
:1030F0002F3F19F4411101C0232F3F5F3630A9F74C
:103100002F3F39F0FC01E20FF11D27FDFA95628394
:10311000089508952091CA043091CB0428173907E7
:1031200071F09093CB048093CA04E091C804F091AD
:10313000C904309721F00084F185E02D09940895A9
:103140002091C6043091C7042817390771F0909375
:10315000C7048093C604E091C804F091C904309775
:1031600021F00680F781E02D09940895E091C804CC
:10317000F091C904309721F00190F081E02D09947D
:1031800080E00895EF92FF920F93CF93DF93C42FC7
:10319000D22FFC0182818823D1F04093C5040E9484
:1031A000F8179093C4048093C30480E28C0F883096
:1031B00008F06DC0C77081E001C0880FCA95EAF7BA
:1031C000DF91CF910F91FF90EF900C948D0480913F
:1031D000C50448134BC08091C3049091C4040E945D
:1031E000E917883C910508F041C0CD17C9F080E28D
:1031F0008C0F883040F4C77081E001C0880FCA95F9
:10320000EAF70E94860480E28D0F883048F481E05E
:103210009D2F977001C0880F9A95EAF70E948D0440
:10322000093319F0E12CF12C03C080E5E82EF12CD4
:10323000802F0E94C904E114F10451F08FE99FE04E
:103240000197F1F700C0000091E0E91AF108F3CF0F
:10325000802F0E94970480E28D0F8830C0F4D770D1
:1032600081E001C0880FDA95EAF70AC080E28C0F8E
:10327000883068F4C77081E001C0880FCA95EAF70A
:10328000DF91CF910F91FF90EF900C948604DF9126
:10329000CF910F91FF90EF900895882311F0FA01DC
:1032A00001C0FB0109941F93CF93DF93FC01E05E03
:1032B000FD4F20816223D1F0EC010E944C30182F89
:1032C0000E944C308F77782F20E8720F08F47FEF40
:1032D000612F8091F1050E94D82B462F282F672F50
:1032E000CE01DF91CF911F910C94C22ADF91CF9133
:1032F0001F910895DF92EF92FF920F931F93CF9348
:10330000DF93EC01FC01E05EFD4F9081692381F1C8
:10331000D090F0050091F1051091EF05E12EF12C10
:103320000E944C30282FC7018C549F4F68E671E0F3
:103330000E941A318E199F0997FD039695958795DE
:10334000959587952370612F289F600D11247D2D01
:10335000802F0E94D82B462F282F672FCE01DF9178
:10336000CF911F910F91FF90EF90DF900C94C22AA4
:10337000DF91CF911F910F91FF90EF90DF90089513
:1033800080E008959091D10492FF0DC0282F2871FC
:10339000283019F4877F846006C0282F24712430D8
:1033A00011F48B7F886093FF0DC0282F287128317E
:1033B00019F4877E846106C0282F2471243111F40A
:1033C0008B7E88612091D20420FF0DC0382F387188
:1033D000383019F4877F816006C0382F3171313061
:1033E00011F48E7F886021FF0DC0282F28712831AD
:1033F00019F4877E816106C0282F2171213111F4D3
:103400008E7E886194FD877E0895F894E82FE2957A
:10341000EF70F0E031A1282F2F7081E090E001C023
:10342000880F2A95EAF7982F9095932391A392A15C
:10343000892B82A378940895CF93DF9382389105E6
:1034400069F1B0F48133910509F46FC048F4893211
:10345000910509F465C08A32910509F46BC08AC0F0
:103460008533910509F457C089339105B9F082C0BD
:10347000833E910571F138F4803E9105B1F0823EB2
:10348000910511F177C0863E9105B9F1873E91050E
:10349000C9F1843E910509F06DC024C02091D1048A
:1034A00020FD53C021FD51C065C08091D10480FD35
:1034B00046C08091D20480FF48C08091D10484FD31
:1034C00050C183EE90E04FC18091D10482FF3AC099
:1034D000F4CF8091D10482FD35C08091D20480FD6B
:1034E00034C0EBCF8091D20481FF35C08091D104EC
:1034F00084FD37C187EE90E036C18091D10483FF0F
:1035000027C0F4CF8091D10483FD22C08091D204E2
:1035100081FD21C0EBCF8091D10485FD1FC021C06A
:103520008091D10485FD1DC019C08091D10486FD14
:103530001BC01DC08091D10486FD19C015C089E350
:1035400090E011C182EE90E00EC180EE90E00BC1E0
:1035500086EE90E008C184EE90E005C189E290E03B
:1035600002C185E390E0FFC08AE290E0FCC081E305
:1035700090E0F9C0811531E5930708F069C0811525
:1035800040E59407F0F09C0174E0369527957A9514
:10359000E1F7922F9370482F437021E030E002C092
:1035A000220F331F4A95E2F73C68392B982F9F7002
:1035B0009695969540E2949FC0011124822B932BFF
:1035C000D2C0883E910568F5803E910508F0CBC0D9
:1035D000883A9105B8F4853A910548F0855AE82F64
:1035E000F0E0E45EFE4F808190E09064BCC08130EA
:1035F000910509F4B3C008F4B4C08430910508F40F
:10360000B0C0B1C08F3B910508F0ABC0885AE82F1D
:10361000F0E0EE0FFF1FE15EFE4F80819181946428
:10362000A2C0811520E2920758F4811531E093077A
:1036300008F099C08D3E910508F493C0906593C041
:10364000811540E4940708F48CC09F70906A8BC089
:10365000811525E5920708F042C0811534E59307EE
:1036600028F0982F8827846F906A7DC0811543E5E4
:103670009407B0F09C012370332741E050E002C072
:10368000440F551F2A95E2F7282F2695269580E2AC
:10369000289F90011124CA01822B932B9A6863C042
:1036A000811522E5920728F4982F8827816F906A68
:1036B0005AC09C012370332741E050E002C0440F00
:1036C000551F2A95E2F7282F2695269580E2289FF8
:1036D00090011124CA01822B932B9C6844C0EC01F9
:1036E000811539E59307A8F48115984528F09C2F9A
:1036F0008827806F906A37C0C11586E5D80788F59E
:103700008C2F0E94C2198F7190E0982F88279062A9
:103710002AC081152AE5920790F48C2F8F700E94A1
:10372000C21994E0D695C7959A95E1F7CF70D0E08D
:10373000DC2FCC27D0699E01282BC90114C09056DC
:103740008115904270F48D2F8F710E94C219282F1D
:103750002F71CE0199279062922B05C081E090E0F5
:1037600002C080E090E0DF91CF910895CF9384E094
:1037700090E00E947530C82F82E290E00E94753080
:103780002C2F30E0A901582BCA01CF91089569EE82
:103790007EEF80E090E00E94B13060E082E090E057
:1037A0000E94933060E083E090E00E94933010929A
:1037B000530510925405109255051092560560E07D
:1037C00084E090E00E94933060E082E290E00E940A
:1037D000933060E085E090E00E94933060E086E006
:1037E00090E00E9493306FEF87E090E00E9493306A
:1037F00040E050E0BA0188E090E00E94A53060E02F
:103800008DE090E00E94933040E050E0BA0188E102
:1038100090E00E94A53060E087E190E00E94933044
:1038200040E050E0BA018CE190E00E94A53060E0F9
:1038300070E080E290E00E94B13040E050E0BA01D8
:1038400088E190E00E94A53040E050E0BA018FE0AE
:1038500090E00E94A53040E050E0BA0183E190E0A2
:103860000C94A53080915205811110925205089553
:1038700080959091510589238093510508959091E9
:10388000510580915005982B9093D7048091520553
:103890008823D9F0892B8093D70480911001882345
:1038A00031F08091D10487FF02C08EE101C086E033
:1038B000E9EDF4E090E0815028F021912223D9F342
:1038C0009F5FF9CF91110E94321C40E250E060E30B
:1038D00075E087ED94E00E943431892B21F180E27C
:1038E000E7EDF4E0A0E3B5E001900D928A95E1F7F1
:1038F000E091C804F091C9043097A9F080911001BB
:10390000882359F08091D10487FF07C08091D704A4
:103910008093D80486E08093D7040280F381E02D61
:1039200087ED94E00994089520912F0580958223D6
:1039300080932F05982F977099F430E0482F082E28
:10394000000C550B2417350759F09091D20492FDC5
:1039500007C08595859585950E94220410922F05B4
:103960000895CF93C091D204C2FB992790F998177C
:1039700099F080FBC2F9C093D2046091D10484E035
:1039800090E00E9493306C2F82E290E00E9493308E
:1039900082E0CF910C94941CCF91089580912E05D4
:1039A0009091FD04891719F08F5F8770FBCF089500
:1039B0000F931F93CF93DF938091FC0482958F70B8
:1039C00009F05DC08091F904882309F458C0809102
:1039D0002E051091FD046091F7047091F804C091D8
:1039E000FA04D091FB0491E06F3F09F090E0292F99
:1039F00006E0811709F443C0209721F07F3F21F0B2
:103A000030E003C031E001C0322F90E030FD34C01F
:103A1000089FF001099FF00D1124DF01A250BB4F58
:103A200011963C911197371327C03C91361324C04F
:103A300012963C91129731111FC013964D915C91D3
:103A400014974C1B5D0B483C5105B0F48091FC046D
:103A50008F7080618093FC04ED5FFA4F80818F70DE
:103A60008061808387EF94E00E94E905DF91CF9128
:103A70001F910F910C94CE1C01968770BACFDF91E5
:103A8000CF911F910F910895CF93DF93EC010E9486
:103A9000C90326E4829FC0011124FC012EE0D29FBD
:103AA000E00DF11D1124EC0FF11DEE0FFF1FE4538B
:103AB000FE4F859194910E941C1ADF91CF91089539
:103AC0009F92AF92BF92CF92DF92EF92FF920F93AD
:103AD0001F93CF93DF93CDB7DEB761970FB6F894FE
:103AE000DEBF0FBECDBF8C0185E0F801DE011D9663
:103AF00001900D928A95E1F7F801E2809091F70428
:103B00006091F8044091FA045091FB04411551056D
:103B100031F06F3F31F481E09F3F19F403C081E041
:103B200001C080E0F82FF1709F2E80FD1AC1F801CE
:103B300030812181C380D48087EFA82E84E0B82E05
:103B4000F090F904F601E41BF50BFF2009F4C6C060
:103B50008091FC04E83CF10508F091C0482F407FBB
:103B600009F050C0621311C093130FC0FE2CE11076
:103B70000CC08F7080618093FC04C5010E94E90530
:103B80008091FC04F801858329C1CD2831F02F3FB5
:103B900031F481E03F3F19F403C081E001C080E0CF
:103BA00080FD03C081E08E2502C080E090E0F82F08
:103BB000F170FF2E80FF1CC080912E054091FD0406
:103BC00056E0841709F4E8C090E0589FF001599F2F
:103BD000F00D1124E250FB4F6181261306C0608175
:103BE000631303C06281E61203C001968770E9CFB8
:103BF000FE2CEE2009F4F2C08091FC0481608093D9
:103C0000FC0449C0621306C0931304C0E11002C053
:103C1000F80186C0C8010E945104882351F1EE20AA
:103C200041F12091FC04822F82958F7090E00297E1
:103C300074F08091F7049091F80498878F83198627
:103C4000DB86CA862C87CE0107960E94E90586E0AE
:103C5000F801A7EFB4E001900D928A95E1F70E9478
:103C6000D81C0AC06217C9F0C8010E945104811112
:103C70001EC0C8010E94E905FF24F394AFC0482F7D
:103C8000407F81F787EF94E00E94E90586E0F50127
:103C900011928A95E9F7F12CA1C09313E5CFE110B9
:103CA000E3CFF8018583C8010E94E90554C0EE20E6
:103CB00001F32091FC04822F82958F7090E002978F
:103CC00034F28091F7049091F8049A8389831B82DF
:103CD000DD82CC822E83CE010196B7CFE83CF10580
:103CE000D0F5FE2CEE2029F2621327C0931325C0D5
:103CF0002091FC0420FD18C0822F82958F70482FE0
:103D000050E04115510581F0F80125834F305105F0
:103D100041F08F5F982F9295907F822F8F70892B23
:103D20008583C8010E94E90586E0F801A7EFB4E0A9
:103D300001900D928A95E1F751C0C8010E9451048B
:103D4000811185CF8091FC0481608093FC04C801BF
:103D50000E94E90543C086E0F50111928A95E9F7D2
:103D60003DC0EE2009F485CFC8010E945104F82E11
:103D7000882309F47ECF86E0F801A7EFB4E0019034
:103D80000D928A95E1F78091F7049091F8040E94D2
:103D9000441D0E94D81C22C03D872E878D859E859C
:103DA0000E94441D292F22952F70223028F49F70E5
:103DB00039F0811105C00BC0243028F49F7049F4FC
:103DC000805E883020F0C8010E94E9059F2CF92C04
:103DD00005C0F8019581907F99F7F9CF8F2D6196F5
:103DE0000FB6F894DEBF0FBECDBFDF91CF911F910C
:103DF0000F91FF90EF90DF90CF90BF90AF909F908A
:103E000008958F929F92AF92BF92CF92DF92EF92DE
:103E1000FF920F931F93CF93DF93CDB7DEB72A970F
:103E20000FB6F894DEBF0FBECDBFAE014F5F5F4F40
:103E30007A018AE0FA0111928A95E9F70DE411E01E
:103E40006A01AA24A394B12CF80180818F3F09F460
:103E500047C0F894E82FE295EF70F0E021A18F7051
:103E6000A50102C0440F551F8A95E2F7CA01922F9F
:103E7000982B91A392A18095892382A3789400C066
:103E8000E2E5F1E021E030E0812C912C41914F3FBF
:103E900089F0A42FA295AF70B0E090968C9190E03D
:103EA0004F7002C0959587954A95E2F780FD02C054
:103EB000C90102C080E090E0882A992A220F331FAE
:103EC00051E0E036F50711F7F80180818F3F11F0DE
:103ED0000E94051AF0EAFA95F1F7F60191828082C4
:103EE0000F5F1F4FF2E0CF0ED11C41E002351407E7
:103EF00009F0AACF4AE050E0B7018AE595E00E94B8
:103F0000343111E0009709F410E0892B89F08AE040
:103F1000F701AAE5B5E001900D928A95E1F781E0FD
:103F2000809359050E94F817909358058093570580
:103F300080915905882391F18091570590915805FA
:103F40000E94E917039750F180915A0590915B0503
:103F5000909369058093680580915C0590915D055B
:103F600090936B0580936A0580915E0590915F0543
:103F700090936D0580936C0580916005909161052B
:103F800090936F0580936E05809162059091630513
:103F9000909371058093700510925905812F2A9690
:103FA0000FB6F894DEBF0FBECDBFDF91CF911F914A
:103FB0000F91FF90EF90DF90CF90BF90AF909F90C8
:103FC0008F900895CF93DF93CDB7DEB762970FB68A
:103FD000F894DEBF0FBECDBF84B7877F84BF0FB616
:103FE000F894A89580916000886180936000109299
:103FF00060000FBE90E080E80FB6F89480936100F7
:10400000909361000FBE85B7806885BF85B78068D3
:1040100085BF80EC99E190936702809366020E94CD
:1040200063150E9409168091E20084608093E2008B
:1040300078948091A2058823A1F01091E9001F7067
:104040009091EC00892F817090FD80E8182B1092E0
:10405000E9008091E80083FD0E943A261F701093CA
:10406000E90082E084BD93E095BD9AEF97BD80930F
:104070006E000DE411E0F2E5EF2EF1E0FF2ED80125
:104080008D918D018F3F11F00E94051AE016F10607
:10409000B1F702E511E0E0E6EE2EE1E0FE2EF801D8
:1040A00081918F018F3F11F00E94051AE016F106F1
:1040B000B1F78AE0E8E6F5E0DF01282F1D922A95A6
:1040C000E9F7EAE5F5E0DF011D928A95E9F780E07E
:1040D00090E00E947D30893E9E4F11F00E94C71BE8
:1040E00082E090E00E947530809372050E94B61BBA
:1040F0009093D2048093D1040E94011FEFEBFDE561
:104100003197F1F700C000000E94011F80916805FF
:1041100080FF08C06FEF7FEF80E090E00E94B13039
:104120000E949F1783E090E00E947530682F70E036
:1041300080E090E00E9447040E9446141092C5055A
:10414000EEEDF5E08EEE95E02FEF3FEF219331930A
:104150008E179F07D9F710920106EAE1F6E08AE28E
:1041600096E02FEF3FEF219331938E179F07D9F7FA
:1041700080E090E00E947D30893E9E4F21F00E94B9
:10418000C71B0E94D62A46E050E06CE170E08EEE3C
:1041900095E00E9465301092C0058091EE058C7FFD
:1041A00011F40E94D62A84E091E09093C904809390
:1041B000C80468E1462E512C72E7672E75E0772E11
:1041C0009924939458E0252E312C8091A2058530B6
:1041D00009F061C040E4F42E00E112E18091A205F3
:1041E000853009F052C08091A205843009F43BC0AB
:1041F00080912E06811105C00E94E30B80E00E9491
:10420000172E21E020932E060E94242E80912E0648
:10421000811105C00E94E30B80E00E94172E31E05F
:1042200030932E061092CC040FB6F894A8954092C5
:1042300060000FBEF092600083B7817F846083BF0F
:1042400083B7816083BF7894889583B78E7F83BF5F
:104250000FB6F894A8958091600088618093600003
:10426000109260000FBE8091A105882309F4B6CF9B
:104270000E94011FE8E6F5E081919191892B09F0F8
:1042800075C26E167F06C1F7A9CF0E9471040E9405
:10429000B61810922E060E94011F882359F08FB77E
:1042A000F8944091CD045091CE046091CF04709168
:1042B000D0048FBFA8E6B5E0E3E7F5E0C12CD12C30
:1042C0000C2DAD90BD90819191918A259B250097F1
:1042D00009F449C110E0EE24E394F12C9C012E2155
:1042E0003F21232B09F439C119870A87AE20BF204B
:1042F00081E0A114B10409F480E08B870E94F817D3
:104300008160782F9D878C8749855A856B858D853F
:104310000E944105F601EE0FFF1FED58FA4F808114
:104320009181E826F926F182E082AB2849F0AE01BE
:104330004F5F5F4F612F802F0E94C42A882E01C0DB
:10434000812CE82CF12C80910106B701680F711DBA
:10435000693071055CF15101AE18BF08B7016E5F9D
:10436000794FA50182E096E00E944131B701665F76
:10437000794FA5018AE096E00E944131A501440FE2
:10438000551FB701660F771F665E794F8AE196E089
:104390000E944131B7016E5E794FA50182E196E03E
:1043A0000E94413188E0881980930106F09001064F
:1043B000AE014F5F5F4F60E0862F8F0D861609F1CB
:1043C00090E0DA017D91AD01272F30E0FC01EF5F35
:1043D000F94FD901AA0FBB1FAA55BE4FAC91A183BB
:1043E000220F331FD901A955BE4F2C912187718B04
:1043F000880F991FFC01EF5FF94F128E118E6F5FCE
:10440000DBCF809301068091EE058C7F8C3609F01E
:10441000C2C0AFEFA00FFF24F394F00E5FEF510F77
:1044200041E0410F511780F48EE08C9DF0018D9D8D
:10443000F00D1124ED55FC4FE50FF11D208130E109
:10444000230F08F42FEF2083212F30E07EE07C9DA6
:10445000C0017D9D900D11248D559C4FFC01E20FF4
:10446000F31F7081B0E26B2F760F08F47FEF70833B
:104470004E3051F0FC01E40FF11D708180E1682F96
:10448000760F08F47FEF708375E0F71609F431C0FA
:10449000EF2CF12C511788F48EE08E9DF0018F9D4A
:1044A000F00D1124ED55FC4FE50FF11D80819DE0CD
:1044B000BC01670F08F46FEF6083EEE0EE9DC00172
:1044C000EF9D900D11248D559C4FFC01E20FF31FC1
:1044D000608170E1670F08F46FEF60834E3049F040
:1044E000FC01E40FF11D60817DE0670F08F46FEFC0
:1044F0006083A01708F04FC0B0E0511780F48EE041
:104500008A9FF0018B9FF00D1124ED55FC4FE50FB4
:10451000F11D50816DE0560F08F45FEF50838EE07F
:104520008A9FF0018B9FF00D1124CF018D559C4F78
:10453000FC01E20FF31F208130E1230F08F42FEF7D
:1045400020834E3041F1FC01E40FF11D20813DE05C
:10455000230F08F42FEF20831EC01F5FEE0CFF1CFB
:104560001E3009F0BBCE8FEFC81AD80A95E0C916E5
:10457000D10409F0A5CE8FEF8E878F87188A0E940D
:10458000F8178160782F9A8B898B4E855F856889B3
:104590008A890E9441050E94242E86E0EBEFF5E017
:1045A000DE01119601900D928A95E1F7E090FD05EC
:1045B000F090FE050091FF05109100061092FD0598
:1045C0001092FE051092FF0510920006E11003C044
:1045D000FF2009F44FC08091F9059091FA050E94DF
:1045E000E9179C019091F505992309F4D5C025316F
:1045F000310508F43FC09F3F19F09F5F9093F50588
:10460000EE2061F00E94012D1E1414F09FEF01C0F6
:1046100091E0899F802D11248093FD05FF2061F09A
:104620000E94012D1F1414F09FEF01C091E0899F9B
:10463000802D11248093FE053091FD053323D1F0A8
:104640002091FE052223B1F045EB3403C001112473
:10465000992319F09093FD0502C09092FD0565EB3A
:104660002603C0011124992319F09093FE0502C07E
:104670009092FE05011103C0112309F44FC08091EF
:10468000F7059091F8050E94E9179C019091F405B7
:10469000992309F486C02135310508F43FC09F3FB6
:1046A00019F09F5F9093F405002361F00E94DF2CC6
:1046B000101614F09FEF01C091E0899F802D112406
:1046C0008093FF05112361F00E94DF2C111614F076
:1046D0009FEF01C091E0899F802D112480930006F7
:1046E0003091FF053323D1F0209100062223B1F051
:1046F00075EB3703C0011124992319F09093FF053E
:1047000002C09092FF0535EB2303C00111249923C9
:1047100019F09093000602C0909200068091FD056A
:1047200081110BC08091FE05811107C08091FF05AA
:10473000811103C08091000681110E947C2DEB82C3
:10474000FC820D831E8386E0FE013196ABEFB5E05F
:1047500001900D928A95E1F70E94B61890917D051F
:10476000891709F432CD80937D052CCD09BD19BD83
:1047700009B400FEFDCF8091D8008F7D8093D800D2
:104780008091E00082608093E0008091E00081FDF4
:10479000FCCF0E94710422CD2B30310508F02DCFC3
:1047A00069CF2B30310508F07CCFB8CFCF92DF92A4
:1047B000EF92FF920F931F93CF93DF938C01C091E1
:1047C00012018DE0C89FC02D1124DDE0DC0FDE3327
:1047D00008F0DDE32091F20531E0230F08F42FEF1C
:1047E00030E040E050E06FEF7FEF80E090E00E942B
:1047F000B7307901CD1708F041C0CC2ED12CF6018D
:10480000E05EFD4F9081809113018923A9F1909181
:10481000C505915097FD15C0492F092E000C550B69
:10482000FA01EB53FA4F8189C813F3CF440F551F98
:10483000FA01EB53FA4F218D328D2E153F0548F7C3
:1048400001C097016091F20541E0640F08F46FEF39
:10485000C9010E94BB2BAC016091EF057091F0057E
:104860008091F105F80109950E94D82B462F282F39
:10487000672FC6010E94C22ACF5FBCCF81E0DD3323
:1048800008F080E0DF91CF911F910F91FF90EF90A2
:10489000DF90CF900895DF92EF92FF920F931F93D6
:1048A000CF93DF938C01C09112018DE0C89FC02D82
:1048B0001124DDE0DC0FDE3308F0DDE36091F2056A
:1048C0006695669521E0620F08F46FEF8091C1054F
:1048D0009091C2050E94BB2BD82ECD17F0F4EC2E80
:1048E000F12CF701E05EFD4F908180911301892347
:1048F00091F06091EF057091F0058091F1052D2DFB
:104900004C2FF80109950E94D82B462F282F672F8E
:10491000C7010E94C22ACF5FE0CF81E0DD3308F0FB
:1049200080E0DF91CF911F910F91FF90EF90DF908A
:1049300008959F92AF92BF92CF92DF92EF92FF9233
:104940000F931F93CF93DF936C01C09112018DE001
:10495000C89FC02D1124DDE0DC0FDE3308F0DDE35D
:104960006091F205669566958091C1059091C205AA
:104970000E94BB2B182F80E4810F0E94072B90E828
:10498000F92EF80E812F0E94072B20E8922E980E08
:10499000CD1700F5AC2EB12CF501E05EFD4F9081F6
:1049A000809113018923A1F06091EF057091F005CA
:1049B0008091F105E12E0C2F292D4F2DF60109953F
:1049C0000E94D82B462F282F672FC5010E94C22A8C
:1049D000CF5FDECF81E0DD3308F080E0DF91CF9163
:1049E0001F910F91FF90EF90DF90CF90BF90AF900D
:1049F0009F9008956F927F928F929F92AF92BF92F5
:104A0000CF92DF92EF920F931F93CF93DF933C01EE
:104A1000C09112018DE0C89FC02D1124DDE0DC0F94
:104A2000DE3308F0DDE36091F20566958091C10503
:104A30009091C2050E94BB2B182FCD1708F044C0DF
:104A40008C2E912CF401E05EFD4F9081809113013A
:104A50008923C1F1F401EE0FFF1FEA55FE4FC0801C
:104A6000D12C80E7C81AD108F401EE0FFF1FE955D9
:104A7000FE4FA080B12CE0E2AE1AB108CC9C9001B0
:104A8000CD9C300D300D1124AA9CC001AB9C900D23
:104A9000900D1124820F931F0E94612B082F6091AB
:104AA000EF057091F0058091F105E12E9501A601C9
:104AB000F30109950E94D82B462F282F672FC40198
:104AC0000E94C22ACF5FB9CF81E0DD3308F080E0D9
:104AD000DF91CF911F910F91EF90DF90CF90BF901A
:104AE000AF909F908F907F906F900895CF92DF92BC
:104AF000EF92FF920F931F93CF93DF936C01C091BE
:104B000012018DE0C89FC02D1124DDE0DC0FDE33E3
:104B100008F0DDE36091F20566958091C105909102
:104B2000C2050E94BB2B182FCD1778F5EC2EF12C67
:104B3000F701E05EFD4F908180911301892319F107
:104B4000F701EE0FFF1FE955FE4F208130E02052A4
:104B50003109F701EE0FFF1FEA55FE4F408150E08B
:104B6000405751096091EF057091F0058091F10572
:104B7000012FF60109950E94D82B462F282F672F69
:104B8000C7010E94C22ACF5FCFCF81E0DD3308F09A
:104B900080E0DF91CF911F910F91FF90EF90DF9018
:104BA000CF9008959091EE059370A1F0811102C00D
:104BB000946007C0803210F09C6703C0880F880F94
:104BC000982B9093EE05109211018091C0058160A1
:104BD0008093C00508959091EE05937059F08093ED
:104BE000EF056093F0054093F1058091C005816069
:104BF0008093C00508958093AC056093AD0524E6CD
:104C000030E042E050E06CEA75E080EA0E94C52F97
:104C100021E0892B09F020E0822F0895EF92FF9286
:104C20000F931F93CF93DF937C018B010E9482151A
:104C3000811119C0E70101151105A1F08091E8006B
:104C400085FD0AC08091E8008E778093E8000E947D
:104C50008215882381F307C089918093F100015068
:104C60001109E9CF80E0DF91CF911F910F91FF9063
:104C7000EF9008951F93CF93DF93CDB7DEB7AA9738
:104C80000FB6F894DEBF0FBECDBFE4EAF5E08CEAC4
:104C900095E02091F10021938E179F07D1F7809125
:104CA000A505833009F461C030F4813071F08230A1
:104CB00009F49BC0B2C08A3009F487C08B3009F474
:104CC0006CC0893009F0A9C020C08091A405813A48
:104CD00009F0A3C08091E800877F8093E80080916D
:104CE000A8059091A905892B21F460E280E895E060
:104CF00003C060E080E090E070E00E944117809186
:104D0000E8008B778093E80088C08091A405813209
:104D100009F083C08091A8059091A905029708F039
:104D20007CC08091E800877F8093E8008091E80054
:104D300082FD05C08091A2058111F8CF6EC020913F
:104D4000F3008091F20090E0922B029731F4809171
:104D5000F100813011F0863021F48091F1008093D0
:104D60007F058091E8008B7754C08091A405813A3B
:104D700009F053C08091A8059091A905892B09F0ED
:104D80004CC08091E800877F8093E8008091E80024
:104D900080FFFCCF8091100137C08091A405813243
:104DA000E1F58091A8059091A905892BB1F5809135
:104DB000E800877F8093E8000E94B5158091A605E2
:104DC000809310010E94710428C08091A405813253
:104DD00021F58091E800877F8093E8000E94B51557
:104DE0008091A70580937E0518C08091A405813A23
:104DF000A1F48091E800877F8093E8008091E8002B
:104E000080FFFCCF80917E058093F1008091E800C7
:104E10008E778093E8000E94B5158091E80083FFAB
:104E2000CEC18091A4059091A505492F50E04A304C
:104E3000510508F0C4C1FA01EE59FF4F0C942E3110
:104E4000803821F0823809F0BAC108C08091A005ED
:104E50009091A105992389F082600FC08091A805E7
:104E60008F70873008F0ABC18093E9008091EB0030
:104E700085FB882780F91092E9009091E800977FE0
:104E80009093E8008093F1001092F10065C1282F03
:104E90002D7F09F094C1882319F0823061F08FC111
:104EA0008091A605813009F08AC1933009F080E035
:104EB0008093A1052EC08091A60581112AC0809102
:104EC000A8058F702FEF280F263008F078C1809347
:104ED000E9002091EB0020FF1CC0933021F4809169
:104EE000EB00806214C09091EB0090619093EB0016
:104EF00021E030E0A90102C0440F551F8A95E2F776
:104F00004093EA001092EA008091EB008860809361
:104F1000EB001092E9008091E800877F20C18111A9
:104F20004EC11091A6051F778091E3008078812BF8
:104F30008093E3008091E800877F8093E8000E94DF
:104F4000B5158091E80080FFFCCF8091E300806878
:104F50008093E300111102C082E001C083E08093DE
:104F6000A2052DC18058823008F029C18091A60584
:104F70009091A7058C3D53E0950779F583E08A83EE
:104F80008AE289834FB7F894DE01139620E03EE071
:104F900051E2E32FF0E050935700E49120FF03C06B
:104FA000E295EF703F5FEF708E2F90E0EA3010F0E7
:104FB000C79601C0C0968D939D932F5F243149F70A
:104FC0004FBF8091E800877F8093E8006AE270E03D
:104FD000CE0101960E944117AEC04091A8055091A4
:104FE000A905292F332723303105A9F068F4213092
:104FF000310509F4F3C02230310509F0E0C08BE33C
:1050000090E0E6E6F4E044C02132310521F122329D
:10501000310571F1D4C0992781309105A1F058F084
:10502000029709F0CCC0E3EBF4E0E4918E2F90E01E
:10503000E3EBF4E02AC0EFEDF4E0E4918E2F90E092
:10504000EFEDF4E022C0EFECF4E0E4918E2F90E07D
:10505000EFECF4E01AC04115510509F4C4C0413029
:10506000510509F0ACC089E090E0E1E9F4E010C03E
:105070004115510509F4BCC04130510509F09FC0EC
:1050800086EB90E0E0E7F3E003C0009709F497C0F7
:105090002091E800277F2093E8002091AA05309115
:1050A000AB058217930708F49C0140E021153105F8
:1050B00089F18091A205882309F43DC08530D9F19A
:1050C0008091E80083FD37C08091E80082FD2FC009
:1050D0008091E80080FFEACF4091F3008091F200D8
:1050E00090E0942B2115310559F08830910540F45A
:1050F00044914093F1003196215031090196F2CF4D
:1051000041E0089709F040E08091E8008E778093B5
:10511000E800CCCF4111CDCF0AC08091A2058823F1
:1051200051F0853041F08091E80083FD04C080910A
:10513000E80082FFF2CF8091E8008B778093E8004F
:105140003EC08038E1F58091E800877F8093E800D9
:105150008091A3058093F1008091E8008E77809381
:10516000E8000E94B5152BC0811129C08091A605C9
:105170009091A7059927029714F58091E800877F01
:105180008093E8001091A6051093A3050E94B51521
:10519000111106C08091E30087FD02C081E001C0CB
:1051A00084E08093A20542E061EC81E00E94D41586
:1051B00042E261EC82E00E94D4158091A2058091C8
:1051C000E80083FF1AC08091E800877F8093E800A1
:1051D0008091EB0080628093EB000FC082E190E051
:1051E000E1EAF4E055CF89E090E0E8E7F4E050CF61
:1051F00080E490E0E6E2F4E04BCFAA960FB6F89494
:10520000DEBF0FBECDBFDF91CF911F91089522E881
:10521000241B08F420E0620F08954095282F429F38
:10522000412D1124842F0895E42FF0E0EE0FFF1F8D
:10523000EA55FE4F9081921B97FD9195292F38E1F9
:10524000239F212D1124620F08950F931F9310E0C7
:10525000F801EE0FFF1FEA55FE4F9081905797FD22
:105260009195000F111FF801E955FE4FE081F0E024
:10527000B097DF01AA0FBB1F8D010E0F1F1F200368
:10528000D001219FB00D1124E8E3F0E0E91BF10902
:1052900097FDF3959F01220F331F89010E0F1F1FEA
:1052A00040039001419F300D11242A0F3B1F37FF0F
:1052B00002C021583F4F220F232F221F330B620FB2
:1052C0001F910F9108950F931F93522F10E0F80133
:1052D000EE0FFF1FE955FE4FE081F0E0B097EE0FB3
:1052E000FF1F9F015203D001539FB00D1124000FE7
:1052F000111FF801EA55FE4F008110E00057110917
:10530000000F111F40039001419F300D11242A0FFF
:105310003B1F37FF02C021583F4F220F232F221F70
:10532000330B620F1F910F9108950F931F93522F0C
:1053300010E0F801EE0FFF1FE955FE4FE081F0E0AD
:10534000B0979F015203D001539FB00D1124000F5D
:10535000111FF801EA55FE4F008110E000571109B6
:1053600040039001419F300D11242A0F3B1F37FF4E
:1053700002C021583F4F220F232F221F330B620FF1
:105380001F910F910895EF920F931F9393E0099F40
:1053900080011124159507956E2D600F1F910F91B7
:1053A000EF900895A22F50E0FA01EE0FFF1FE9558C
:1053B000FE4F9081905297FD9195440F551FFA0131
:1053C000EA55FE4F3081232F30E02A1B3109290F87
:1053D000311D97FD3A95620F0895E42FF0E0EE0F2E
:1053E000FF1FE955FE4F6081621B0895E42FF0E036
:1053F000EE0FFF1FEA55FE4F6081621B0895622F7A
:105400000895E42FF0E0EE0FFF1FEA55FE4F4081B4
:1054100034EE439F412D1124E82FF0E050E0445E2C
:105420005F4FDA01A21BB1099D01B7FF03C031959F
:105430002195310993E0220F331F9A95E1F7AF01CF
:10544000421B530B9A0157FF02C020E030E0582F57
:10545000259F212D1124822F0895FC019B01009787
:1054600021F477FF2BC080E80895AC0197FF04C0BA
:1054700044275527481B590BB901640F751F37FD89
:105480000CC0241B350BC901A5E0880F991FAA95F4
:10549000E1F70E941A3180E20CC0CB0165E0880F71
:1054A000991F6A95E1F7BA01621B730B0E941A31CA
:1054B00080E6861BF7FF03C08195089580E008957C
:1054C000EF920F93CF93DF93D72FC82FC9010E19F7
:1054D000BA010E942D2A602F681B7D2F8C2FDF912F
:1054E000CF910F91EF9008950F93CF93DF93D72F24
:1054F000C82FC901BA010E942D2A682F600F7D2F85
:105500008C2FDF91CF910F910895EF920F931F93FE
:10551000CF93DF93D62FC72F182FC9010E19010F74
:10552000BA010E942D2A081B202F219F212D112412
:10553000822F6D2F7C2FDF91CF911F910F91EF90D4
:105540000895FF920F931F93CF93DF93F62ED72FDB
:10555000182FC901C12FC01BBA010E942D2A982FF4
:10556000990F890FC81B2C2F219F212D1124822FC9
:105570006F2D7D2FDF91CF911F910F91FF90089597
:105580000C94F5130C94B2132EE0829FC0011124E9
:10559000FC01E05AFE4FE60FF11D80818F3F21F0A4
:1055A000FA01808381E0089580E00895EEEEF5E051
:1055B00085E280838091190190911A01A0911B01CD
:1055C00081839283A3838FE784838FEF858346E073
:1055D00050E06CE170E0CF010E9483301092C00572
:1055E0000895EF92FF920F939701201B31092F3FEF
:1055F000310519F010F02FEF30E02095382F320FE1
:1056000008F43FEF832F0F91FF90EF900895482FFC
:10561000982F46FD9095E92FEF739F7046FD9F5F91
:10562000E295EF70EE0FF0E0E35AFD4F2181299FE4
:10563000802D212D112482958F702295207F822B21
:105640003081982F930F892F47FD819580580895B9
:105650000F931F93CF93DF93D62F072F182FC42FAD
:10566000822F0E94072BEC2FF0E0EE0FFF1FEA5570
:10567000FE4F90819058890F87FD8195880F682F84
:105680002CE0629F612D11246D0F702F812FDF910F
:10569000CF911F910F9108954091150150911601DE
:1056A00025E038E0429FC001439F900D529F900D2E
:1056B0001124875E994C9093160180931501890FF0
:1056C0000895BC018230910508F40895613E8EE191
:1056D000780748F49B0195E0369527959A95E1F770
:1056E00048E0420F01C04FEF91E0242F30E0290F36
:1056F000311D35952795229FF001239FF00DF00D68
:1057000011246E177F0718F44FEF420F04C02F3F8C
:1057100039F091E0920F491740F78FEF890F089504
:105720008FEF08950F93CF93DF93D72FC82F47FDA7
:105730004195E8E3F0E0CF01841B910947FD939583
:10574000889FB001899F700D700D1124229FC001A8
:10575000239F900D900D1124860F971F0E94612B9F
:10576000682F660F860F682F600F7D2F8C2FDF91BB
:10577000CF910F91089520E030E0869F212D969FD4
:10578000200D311D1124C90108952091F20530E149
:10579000230F08F42FEF60E1822F90E00E94BB2BD3
:1057A000BC0188EB9BE00E94EC2F80E090E0089524
:1057B000CF92DF92EF92FF920F931F93CF93DF93DD
:1057C000F62E472FE82FF0E0711106C0ED51FB4F88
:1057D0008491782F682F73C0272F30E0ED51FB4F55
:1057E000E491FE2F0E2F10E056E0659FC0011124BA
:1057F000CFEFD0E0BE010E94EC2F5BEA5603C00160
:10580000579F900D11248F0D911D8F0D911D982F75
:10581000990F980F7E01E21AF30AE09ED001E19EF3
:10582000B00DF09EB00D11248B2F499FA0011124C3
:10583000452F55277E01E41AF50AE09EA001E19E5E
:10584000500DF09E500D11246E01C91AD108C29E50
:105850007001C39EF00CD29EF00C11242F2D332723
:10586000C21BD30BC09F9001C19F300DD09F300D44
:105870001124932F6230710591F048F46115710580
:10588000E1F061307105B9F49E2FE52F16C0643048
:10589000710569F040F06630710579F00CC09E2FFB
:1058A000EB2F832F0AC0EB2F8F2F952F06C09B2F36
:1058B0008E2FE32F02C09B2F852F7E2F692FDF9124
:1058C000CF911F910F91FF90EF90DF90CF900895AF
:1058D0008D3E39F49091FE0597FF35C01092FE057C
:1058E00059C08E3E29F49091FE051916BCF32BC0C9
:1058F0009091FD058F3E29F497FF25C01092FD057C
:1059000049C0803F19F41916CCF31DC09091FF05D2
:10591000893F29F41916BCF41092FF053BC08A3F59
:1059200019F497FF10C0F8CF8B3F39F4909100061F
:1059300097FF09C0109200062DC08C3F21F4909172
:1059400000061916BCF39FE0980F983080F421E010
:1059500030E0A90102C0440F551F9A95E2F7CA0131
:1059600080959091FC0589238093FC0513C08D3FA1
:1059700021F48091F6058E7F0BC08E3F21F480913B
:10598000F6058D7F05C08F3F29F48091F6058B7F4A
:105990008093F6058091FD05811106C08091FE057A
:1059A000811102C01092F5058091FF05811106C09A
:1059B00080910006811102C01092F4050895809133
:1059C000F60580FD16C081FD16C082FD18C08091CD
:1059D000F405882391F0883290F428E0829FC0017A
:1059E000112468E270E00E941A31862F672B29F09B
:1059F00007C082E0089584E0089581E0089588E07A
:105A000008958091F60580FD14C081FD14C082FDCB
:105A100016C08091F505882381F08E3180F420E551
:105A2000829FC00111246EE170E00E941A31862F1E
:105A3000089584E1089588E2089588E0089580E556
:105A400008958D3E21F40E94012D819504C08E3E63
:105A500029F40E94012D8093FE0508958F3E21F4C4
:105A60000E94012D819504C0803F29F40E94012DE0
:105A70008093FD050895893F19F40E94DF2C05C02D
:105A80008A3F31F40E94DF2C81958093FF050895B1
:105A90008B3F21F40E94DF2C819504C08C3F29F4B8
:105AA0000E94DF2C8093000608959FE0980F9830A5
:105AB00078F421E030E0A90102C0440F551F9A9507
:105AC000E2F7CA019091FC05892B8093FC050895AB
:105AD0008D3F21F48091F60581600BC08E3F21F44B
:105AE0008091F605826005C08F3F29F48091F6050C
:105AF00084608093F60508950E94F8172091FD05B3
:105B0000211104C02091FE05222321F09093FA0573
:105B10008093F9052091FF05211104C02091000612
:105B2000222321F09093F8058093F705E091C804B3
:105B3000F091C904309749F082E08093FB0504801E
:105B4000F581E02D8BEF95E009940895EEEEF5E0F8
:105B5000248130E1231B08F420E024838091C005D8
:105B600081608093C0050895EEEEF5E0248130E178
:105B7000230F08F42FEF24838091C0058160809368
:105B8000C0050895EEEEF5E0438120E1421B08F4E4
:105B900040E08181628190E00C94EB25EEEEF5E02F
:105BA000438120E1420F08F44FEF8181628190E050
:105BB0000C94EB25EEEEF5E0628120E1621B08F427
:105BC00060E08181438190E00C94EB25EEEEF5E0FE
:105BD000628120E1620F08F46FEF8181438190E0E0
:105BE0000C94EB25EEEEF5E0818190E0438162813B
:105BF00008970C94EB25EEEEF5E0818190E043816F
:105C0000628108960C94EB258091EE058695869529
:105C1000815009F48FE10C94D2258091EE05869590
:105C200086958F5F803208F081E00C94D2258093B6
:105C300018018091EE058370809317010E940F1464
:105C400083E08093110108958F929F92AF92BF924B
:105C5000CF92DF92EF92FF921F93CF93DF93409109
:105C60002A0650912B0660912C0670912D062FB7B5
:105C7000F8948091CD049091CE04A091CF04B0917E
:105C8000D0042FBF841B950BA60BB70B2FB7F8942E
:105C9000C090CD04D090CE04E090CF04F090D0041A
:105CA0002FBFC0922A06D0922B06E0922C06F092CB
:105CB0002D0610910106E1E0F6E0212F30E04FEFD4
:105CC0005FEF60E070E0481B590B6A0B7B0B13170A
:105CD00099F0C18DD28D4E01A12CB12C48155905DA
:105CE0006A057B0510F4215004C0C80FD91FD28F5C
:105CF000C18F3F5F3296EBCF2093010680912E0635
:105D0000811108C0C091EE058C2F837019F0C695E3
:105D1000C69501C0C0E0809111018130F1F030F0F2
:105D20008230B9F1833009F442C06CC01092120184
:105D3000C092C105D092C205E092C305F092C4059D
:105D400089E2E1E0F6E0A5ECB5E001900D928A95DC
:105D5000E1F781E08093110155C08C2F0E94E30B85
:105D6000CC2309F44FC00E94B61881FF4BC02FEF1F
:105D70004FEF6FEF88E290E0DF91CF911F91FF909E
:105D8000EF90DF90CF90BF90AF909F908F900C944A
:105D9000C22A8C2FDF91CF911F91FF90EF90DF905F
:105DA000CF90BF90AF909F908F900C94172E8091C2
:105DB000C005882351F046E050E06CE170E08EEEC3
:105DC00095E00E9483301092C0054091C10550912A
:105DD000C2056091C3057091C4052FB7F8948091F6
:105DE000CD049091CE04A091CF04B091D0042FBFE8
:105DF000841B950BA60BB70B4097A105B10510F0BE
:105E000010921101DF91CF911F91FF90EF90DF90E1
:105E1000CF90BF90AF909F908F9008951092B9004F
:105E20008CE08093B80008959F92AF92BF92CF927A
:105E3000DF92EF92FF920F931F93CF93DF93B82ED1
:105E4000EB010E94F8176C01C431D10558F0CF3F27
:105E50008FEFD80759F0CE0164E170E00E94EC2F7B
:105E60007B0107C0EE24E394F12C03C025E0E22E71
:105E7000F12C84E8A82E94EA992E1092BC009092FE
:105E8000BC000E94F8178C018091BC0087FD08C0FF
:105E90000E94F817801B910B8E159F05A8F32AC04E
:105EA0008091B900887F883041F08091B900887F67
:105EB000803119F00FEF1FEF1FC0B092BB00A0920E
:105EC000BC000E94F8178C018091BC0087FD08C0BF
:105ED0000E94F817801B910B8E159F05A8F30AC02E
:105EE0008091B900887F883111F0803419F700E083
:105EF00010E00EC00EEF1FEFCF3F8FEFD80709F471
:105F0000BCCFC6010E94E9178C179D0708F4B5CFD6
:105F1000C801DF91CF911F910F91FF90EF90DF901B
:105F2000CF90BF90AF909F9008950F931F93CF9302
:105F3000DF93EB018093BB0084E88093BC000E9458
:105F4000F8178C018091BC0087FD0EC0CF3F8FEF0A
:105F5000D807C1F30E94F817801B910B8C179D077F
:105F600088F38EEF9FEF0CC02091B900287F81E06D
:105F700090E0283211F480E090E0919581959109AC
:105F8000DF91CF911F910F910895CF92DF92EF9201
:105F9000FF920F931F93CF93DF936B018A017901D7
:105FA000B9010E94142FE6010C0D1D1DC017D10769
:105FB00061F424E92093BC00DF91CF911F910F91F0
:105FC000FF90EF90DF90CF90089597FDF2CFB7014B
:105FD00089910E94952FEACFAA1BBB1B51E107C0F4
:105FE000AA1FBB1FA617B70710F0A61BB70B881F69
:105FF000991F5A95A9F780959095BC01CD010895F8
:106000008F929F92AF92BF92CF92DF92EF92FF92C8
:10601000CF93DF93EC01688179818A819B8161153F
:1060200071058105910521F464E279ED8BE597E036
:106030002DE133EF41E050E00E94B73049015A01B1
:106040009B01AC01A7EAB1E40E94D6306B017C0150
:10605000ACEEB4EFA50194010E94E430DC01CB0169
:106060008C0D9D1DAE1DBF1DB7FF03C00197A1097B
:10607000B04888839983AA83BB839F77DF91CF91B0
:10608000FF90EF90DF90CF90BF90AF909F908F9058
:1060900008950E940030089580E091E00E94003051
:1060A0000895A0E0B0E08093000190930101A093D7
:1060B0000201B09303010895FB01DC0102C00590C9
:1060C0000D9241505040D8F70895DC01CB01FC01FE
:1060D000F999FECF06C0F2BDE1BDF89A319600B441
:1060E0000D9241505040B8F70895F999FECF92BDF6
:1060F00081BDF89A992780B50895A8E1B0E042E003
:1061000050E00C946730DC01A40FB51F41505040A3
:1061100048F0CB01840F951F2E910E94943041507E
:106120005040D0F70895262FF999FECF92BD81BD3A
:10613000F89A019700B4021639F01FBA20BD0FB6C5
:10614000F894FA9AF99A0FBE08950396272F0E94A1
:1061500094300E949330252F0E949430242F0C9469
:1061600094300196272F0E9494300C949330052E82
:1061700097FB1EF400940E94CE3057FD07D00E947A
:10618000E93007FC03D04EF40C94CE305095409586
:10619000309521953F4F4F4F5F4F089590958095D3
:1061A000709561957F4F8F4F9F4F08950E940B31DF
:1061B000A59F900DB49F900DA49F800D911D11245B
:1061C0000895B7FF0C94D6300E94D630821B930BF3
:1061D0000895A1E21A2EAA1BBB1BFD010DC0AA1F28
:1061E000BB1FEE1FFF1FA217B307E407F50720F040
:1061F000A21BB30BE40BF50B661F771F881F991FBB
:106200001A9469F760957095809590959B01AC0103
:10621000BD01CF010895A29FB001B39FC001A39F0C
:10622000700D811D1124911DB29F700D811D1124CF
:10623000911D089597FB072E16F4009407D077FD63
:1062400009D00E94EC2F07FC05D03EF49095819573
:106250009F4F0895709561957F4F0895EE0FFF1F32
:106260000590F491E02D0994FB01DC0104C08D91AF
:106270000190801921F441505040C8F7881B990BB8
:106280000895FB01DC0102C001900D924150504085
:08629000D8F70895F894FFCF40
:10629800010000001C13711352134E134A131B13F1
:1062A800010300FF003905FFFF00FFFF818283E241
:1062B80000E900EA00B500B600B700CD008301CCC4
:1062C800008A019201940121022302240225022658
:1062D8000227022A02B300B4006F007000F5F4F13F
:1062E800333267F7F6F030313497969495939237B6
:1062F8000D0C0B0A090807060504030201001B1A06
:10630800191817161514131211100F0E2827262501
:1063180024232221201F1E1DFF1C34333231302F2D
:106328002E2D2C2B2A29FFFF3C3B3AFFFF39FFFF7C
:10633800FF383736FF35D800C000B000A000900005
:106348008000700060005000400030002000100005
:106358000000DC10C810B810A81098108810781029
:106368006810581048103810281018100410D61843
:10637800BC20AC209C208C207C206C205C204C20F5
:106388003C202C201C200620D230B430A43094307D
:1063980084307430643054304430343014300A302F
:1063A800DE40CA40B640A24066402A40164002403D
:1063B80001010101010101010101010101010104C2
:1063C800040404040404040404040401010404048B
:1063D800040404040404040401010404040404047B
:1063E8000404040401010101010401010100313127
:0663F800295A1B750A0082
:00000001FF
